:020000040000FA
:1000000049288207003400340034013400340034BD
:1000100000340A34003400340034643400340034D2
:100020000334E8340034003427341034003401340D
:100030008634A03400340F344234403400349834D1
:10004000963480348207073406340534043403348C
:1000500002340134003482075334563433344F347D
:10006000523441340034423461346E3464342034C8
:10007000003455347034643461347434653400347D
:1000800049346E3469347434423461346E346434C7
:1000900000348B0107309F009801831698018C0172
:1000A0009F018113FF30850086018312A901AA01F7
:1000B000AB01AC01AD015D225D2277229722373082
:1000C0008400F0017B23C601CA010508C500033086
:1000D0004505C400451EE721D1015330DC00003046
:1000E000CD000301CE210430F0009323D200A920DB
:1000F000C321222307309D2207239C23E2225C2276
:100100005C221A214A1E86288F208128C6188A2838
:10011000FE208C28B520D420E2225C228128FF30EA
:100120005C078400C6189A288003801FA0280D3021
:100130008000A028800A0E300002031CA028800145
:10014000222307309D2207239C23A920E2225C2240
:1001500008005C08FF3E8400053000070007000728
:100160000007F000840A7B230800CC015C088400AF
:100170002E0880070330C800CE20840384032F0894
:1001800080070230C800CE20840330088007840A2C
:10019000031CCB28800A3108800708004C0D840A14
:1001A0008007C80BCE28080003305C0784000330AA
:1001B0000002031CFD28031DF02884039330000275
:1001C000031CFD28031DF028840387300002031C54
:1001D000FD28031DF028840300300002031CFD28C5
:1001E0005C08840000308000840A87308000840A24
:1001F00093308000840A0330800008000E21B5206F
:1002000003305C078400801F0C2980018403800177
:1002100084038001840380010E210800AE09AF0928
:10022000B009B109AE0F1929AF0F1929B00F19295B
:10023000B10A08004C210508C500B1230508450690
:10024000031D1A2903304505C300440603191A2962
:100250000310C40D4308C40644080239C70046060B
:10026000C601C4183B294308C400D00350181A29FA
:10027000D0181A2944290230C6004308C400D00A05
:1002800050181A29D0181A294308C400C5194A2938
:100290004A164B294A120800CA18AC29051DAD2977
:1002A000051A6929851D8E292030CB004A10A82304
:1002B000051A6729851D8E29051DAD29CB03031D50
:1002C00057290130CE210430CB004A145729013080
:1002D0008A294A1E6F29851DAC29CA01AC298519B6
:1002E000AC29CA1977292030CB004A10CA15A82397
:1002F00085198929051E8E29CB0303198229CA195C
:10030000AC297729CA11FF30CE210430CB004A1422
:100310007729FF304A18AB29CE21AB294030CB00DA
:10032000A823051AAC298519AC29CB03031D9029F4
:100330004A1EA4295F2322230D309D229C232223C1
:1003400014309D229A23AA29662322230D309D2250
:1003500007239A23E222CA010800A823051ECA1611
:10036000051DAD29CA1EB629C321BF29511CBC29B0
:1003700051105330DC00BF2951145830DC00CA0141
:10038000E2225C22AC295308D8005408D900550851
:10039000DA005608DB005208D70008004D0707397D
:1003A000CD002220CE00D621E22208000430C80071
:1003B000313084004D08CC000310CC0DCC0D4C081E
:1003C000012080008403CC0AC80BDF290800CA146E
:1003D0008030D3009630D4009830D5000030D6005D
:1003E000E2225C221A21B101B001AF010530AE005A
:1003F0004519FC298030AE000000C618002A0E21E5
:100400002E08B707031C092AB80F092AB90F092AB1
:10041000BA0A2F08B807031C102AB90F102ABA0A03
:100420003008B907031C152ABA0A3108BA07051E95
:10043000F129F001373084007223CA100800A901A5
:10044000AA01AB01AC01AD012030B4003708BB00FC
:100450003808BC003908BD003A08BE005C088400BA
:1004600003103B1C4D2A0008AA07031C3C2AAB0FB3
:100470003C2AAC0F3C2AAD0A840A0008AB07031CD7
:10048000442AAC0F442AAD0A840A0008AC07031CB6
:100490004A2AAD0A840A0008AD07AD0CAC0CAB0CBF
:1004A000AA0CA90CBE0CBD0CBC0CBB0C5C08B40B9C
:1004B0002F2A0130AD0008001F22293084000008D7
:1004C000B6000830B500B60C031C6A2A861506155E
:1004D00006116D2A861106150611B50B632A840ACA
:1004E0002E300402031C5F2A861786130800A523FA
:1004F000033086000616A523061203308600061672
:10050000A8230612033086000616A823061202301E
:1005100086000616AB23061220303D2308303D230B
:1005200001303D2306303D230E303D2308000030CE
:100530009D229A2380303D230800CF002B20FF39D5
:100540000319A62A4123CF0A4F089E2A080020300B
:10055000B200A401A501A601A701A8015C088400BE
:100560000008A000840A0008A100840A0008A20074
:10057000840A0008A3000310A00DA10DA20DA30D75
:1005800003182014A40DA50DA60DA70DA80DB203E8
:10059000031DCB2A080024308400D722840AD722E6
:1005A000840AD722840AD722840AD722BB2A03309E
:1005B0000007B300B319800030300007B300B31B4D
:1005C00080000800A72202303D23270E0F39303E5D
:1005D000412327080F39303E4123260E0F39303E84
:1005E000412326080F39303E4123250E0F39303E76
:1005F000412325080F39303E4123240E0F39303E68
:10060000412324080F39303E41231E230800A40152
:10061000A501520851185708CC00CC0A0A304C02E8
:10062000031C152BA400A50A172B4C08A4002508B1
:10063000303E41232408303E4123080080304E04E0
:100640003D23080001303D23080086018316083051
:100650008600831206138616FF30C10006160608B0
:10066000C000061200000000061600000612C103BA
:1006700003193C2BC0192E2B0800BF00C90106131B
:10068000442BBF004914061725238601831600302A
:10069000860083128612061349180617F030860565
:1006A0003F0E0F398604061600000612F03086054C
:1006B0003F080F39860406160000061208000430B1
:1006C000F00052085118570884230800FF305C07D7
:1006D00084000008CC0005304C074C074C074C0741
:1006E000F000840A0430C80000088423840AF00A59
:1006F000C80B742B08000430C80093238000F00A54
:10070000840AC80B7D2B080083169A0070089B0092
:100710001C1555309D00AA309D009C149C188E2BF2
:100720001C1183120800831670089B001C141A0801
:10073000831208009F239F239F239F230800A22347
:10074000A2230800FF30C100B32B8030C100B32BBF
:100750004030C100B32B2030C100B32B1030C1009A
:10076000B32B0230C100FF30C200C20BB52BC10B4E
:04077000B32B08009F
:084000005700330043004400A7
:02400E00303F41
:10420000DF006500DC001700020050009E001B006C
:104210000000400052003600000000006C006B00FF
:104220000000A0005B009A000000E0008900D600BA
:10423000000080001F0014000100A0005900410090
:104240000100100009007C00010060002900AC00A2
:104250000100E0004400A3000000C8002200560056
:1042600000003800FF004A000000B800CD00330015
:1042700000005800F10006000000000000000000EF
:00000001FF
